:0400000010EF00F00D
:08000800FACF7FFFBCEF0DF001
:10001800D8CF64FFB6EF0DF00AEE20F01FEE64F0C3
:10002800C6EC28F000EE11F010EE13F0C6EC28F044
:1000380000EE74F011EE00F0C6EC28F05FEF0EF061
:100048000001CF6BD06BD16BD26B2B0ED36F0A0E26
:10005800D46F76EC1FF0006E00C002F0036A035004
:100068000210D8B4000CEDCBE8FF040AD8B405D0D0
:10007800EDCBE8FF060AD8A40AD029CCE8FF550A38
:10008800D8A405D02ACCE8FFAA0AD8B406D0000123
:10009800826B836B846B856B44D0F1CB00F00001DD
:1000A80000C082F0836B846B856B080EF2CB00F086
:1000B800016A026A036A91EC28F000EE82F00050AF
:1000C800EE260150EE220250EE220350ED22ED52B0
:1000D800ED52100EFDCB00F0016A026A036A91EC42
:1000E80028F000EE82F00050EE260150EE22025079
:1000F800EE220350ED22ED52ED52180EFECB00F029
:10010800016A026A036A91EC28F000EE82F000505E
:10011800EE260150EE220250EE220350ED22ED525F
:10012800ED5282C0CFF083C0D0F084C0D1F085C03A
:10013800D2F000012B0ED36F0A0ED46F76EC1FF0AD
:10014800006E00C002F0036A03500210D8B4000C1D
:100158002BCAE8FFE90AD8B405D02BCAE8FFEB0A96
:10016800D8A4000C0AEE36F0EF50D8A4000C37CA19
:10017800E8FF020AD8A4000C40CAE8FFF80AD8A48D
:10018800000C3DCA79F03CCA78F078C000F079C01C
:1001980001F0050ED89000360136E82EFBD7000690
:1001A800010E0122090E026ED89001320032022E91
:1001B800FBD700500001BA6F0150BB6FBC6BBD6B21
:1001C8003ACA01F0006A000E01BEFF0E026E036E0D
:1001D80039CAE8FF0024046E000E0120056E000EE7
:1001E8000220066E000E0320076E00EE82F0045017
:1001F800EE260550EE220650EE220750ED22ED5273
:10020800ED5242CA01F0006A41CAE8FF0024046EB8
:10021800000E0120056E066A05BE06060650076E2A
:1002280004C0BEF005C0BFF006C0C0F007C0C1F0F2
:100238003BCA2AFABEC004F0BFC005F0C0C006F031
:10024800C1C007F02ACA00F0016A026A036ACFEC4B
:1002580027F082C0E8FF0024E8CF7EF083C0E8FFE3
:100268000120E8CF7FF084C0E8FF0220E8CF80F0CB
:1002780085C0E8FF0320E8CF81F038CA29FABA0E12
:10028800E96E000EEA6E0001EE507E25E8CF7AF0A6
:10029800EE507F21E8CF7BF0EE508021E8CF7CF054
:1002A800ED508121E8CF7DF0ED52ED52010CBE00FA
:1002B8000001C36BC46BC56BC66BBEC0D9FFBFC0A2
:1002C800DAFFC051D8A409D000EE0CF0D950E926C5
:1002D800DA50EA22EE6AED6AC9D10001C005D8B445
:1002E800BCD10001C051020AD8A4C0D1ACD17EC093
:1002F80004F07FC005F080C006F081C007F000EE72
:100308000CF0D950E926DA50EA22EECF00F0EDCF12
:1003180001F0040E026ED89001320032022EFBD793
:10032800026A036A00500426015005220250062280
:100338000350072200EE0CF0D950E926DA50EA22E1
:10034800EECF00F0EDCF01F00F0E0016000E0116F3
:10035800050ED89000360136E82EFBD700C0C1F054
:1003680001C0C2F0D9CFBEF0DACFBFF0000107500C
:10037800C61908E10650C51905E10550C41902E17E
:100388000450C319D8B41ED004C0C3F005C0C4F0CB
:1003980006C0C5F007C0C6F0C3C0CFF0C4C0D0F0D7
:1003A800C5C0D1F0C6C0D2F02B0ED36F0A0ED46FE1
:1003B80076EC1FF0006E00C002F0036A03500210D2
:1003C800D8B4000CBEC0D9FFBFC0DAFF00010AEEE6
:1003D8002BF0C151E926C251EA22EF50D8B42ED1F0
:1003E8000AEE2BF0C151E926C251EA22EF50E50A84
:0803F800D8B424D100010AEE83
:100400002BF0C151E926C251EA22EF502E0AD8B48E
:1004100019D100010AEE36F0C151E926C251EA2293
:10042000EF501A0BD8A40ED1F36AF3500001C12586
:10043000006E000EC221016E2B0E0024E16E0A0E2A
:100440000120E26EF350D924E96E000EDA20EA6E44
:10045000E7CFEFFFF32A0A0EF364E7D7F350D9246E
:10046000E96E000EDA20EA6EEF6AF3500AEE47F00A
:10047000E926000EEA22EF50006E00C002F0036A87
:1004800000EE10F0D950E926DA50EA2202C0EEFF61
:1004900003C0EDFF0AEE48F0C151E926C251EA223D
:1004A000EF50016E006A00EE10F0D950E926DA50E4
:1004B000EA220050EE260150ED2200EE10F0D95055
:1004C000E926DA50EA22EE06010EED22090E006E50
:1004D00000EE10F0D950E926DA50EA22002804D0C4
:1004E000D890EC32ED52EF32E82EFAD70AEE49F00E
:1004F000C151E926C251EA22EF50006E00C002F05D
:10050000036A070ED89002360336E82EFBD700EEBA
:1005100010F0D950E926DA50EA220250EE260350B4
:10052000ED220AEE45F0C151E926C251EA22EF5010
:10053000006E0AEE46F0C151E926C251EA22EF50A0
:10054000036E00C002F000EE16F0D950E926DA5032
:10055000EA2202C0EEFF03C0EDFF0AEE4AF0C151ED
:10056000E926C251EA22EF50006E016A026A036A6C
:10057000080E91EC28F000C0C7F001C0C8F002C01E
:10058000C9F003C0CAF00AEE49F0C151E926C251D0
:10059000EA22EF50006E016A026A036AC751002620
:1005A000C8510122C9510222CA510322080E91ECFE
:1005B00028F000C0CBF001C0CCF002C0CDF003C0E9
:1005C000CEF00AEE48F0C151E926C251EA22EF50BE
:1005D000006E016A026A036ACB510026CC510122E7
:1005E000CD510222CE510322080E91EC28F00AEEE2
:1005F00047F0C151E926C251EA22EF500024046EAF
:10060000000E0120056E000E0220066E000E032073
:10061000076E00EE12F0D950E926DA50EA2204C043
:10062000EEFF05C0EEFF06C0EEFF07C0EDFFED5286
:10063000ED5200EE0EF0D950E926DA50EA22EE6AC9
:10064000ED6A010C0001C051020AD8A40AD000EEE4
:100650000CF0D950E926DA50EA22EE06000EED5AE7
:1006600009D000EE0CF0D950E926DA50EA22EE2A41
:10067000000EED2278C000F079C001F000EE0CF021
:10068000D950E926DA50EA22EECF02F0EDCF03F09E
:100690000150035C02E10050025CD8A02CD600EEB1
:1006A00010F0D950E926DA50EA22EE6AED6A000C21
:1006B000BA000001BC6BBD6B000100EE16F0BA5130
:1006C000E926BB51EA22D890BC35006EBD35016EDB
:1006D0002B0E0024E16E0C0E0120E26EEECFE6FF41
:1006E000EDCFE5FFBAC0C7F0BBC0C8F021D8006E9F
:1006F00000C002F0036A03500210D8B4000C0001DD
:10070000BC4BBD2B010EBD5D7F0ED8B4BC5DD8A027
:10071000D3D7000110EE16F0BA51E126BB51E22208
:100720000FEE29F0E6CFEEFFE5CFEDFF010CC7009D
:10073000C7C0E1FFC8C0E2FF00EE0EF0E150E926BD
:10074000E250EA22EE2A000EED2229CA02F0036AE4
:1007500000EE0EF0E150E926E250EA22EECF00F082
:10076000EDCF01F012EC28F001500010D8A4010CDC
:1007700082C0CBF083C0CCF084C0CDF085C0CEF079
:1007800000EE16F0E150E926E250EA22EECF00F04A
:10079000EDCF01F001C000F0016A026A036A0001B6
:1007A0000050CB270150CC230250CD230350CE2341
:1007B00000EE16F0E150E926E250EA22EECF00F01A
:1007C000EDCF01F00050C96FCA6BE1CFC7F0E2CFA7
:1007D000C8F0D890C937CA37CBC0CFF0CCC0D0F062
:1007E000CDC0D1F0CEC0D2F02B0ED36F0A0ED46F95
:1007F00076EC1FF0006E00C002F0036A0350021096
:10080000D8B4000C00010AEE2BF0C951E926CA51F8
:10081000EA22EF50006E0AEE2CF0C951E926CA51C7
:10082000EA22EF50036E00C002F000EE16F0C7514E
:10083000E926C851EA2202C0EEFF03C0EDFF010C19
:10084000D000090ED2C000F0D3C001F0D4C002F035
:10085000D5C003F086EC28F000C0E4F001C0E5F05C
:1008600002C0E6F003C0E7F00001D251DC6F010ED8
:10087000D315DD6FDE6BDF6BD0C0D9FFD1C0DAFFDF
:10088000D651DC25006ED751DD21016E000EDE2130
:10089000026E000EDF21036E000E035C08E1000E05
:1008A000025C05E1020E015C02E1000E005CD8B0C2
:1008B0000BD0D651E06FD751E16FE26BE36BD86B91
:1008C000D96BDA6BDB6B25D0DC0EE96E000EEA6EBD
:1008D0000001EE500008E06F020EEE54E16F000ED2
:1008E000EE54E26F000EED54E36FED52ED52D6C0C0
:1008F00000F0D7C001F0026A036AE051005CD86FD3
:10090000E1510158D96FE2510258DA6FE3510358AF
:10091000DB6F0001D890E435006EE535016E2B0EDB
:100920000024E16E0C0E0120E26E00EE16F0D950AC
:10093000E926DA50EA22E6CFEEFFE5CFEDFF00EE42
:100940000EF0D950E926DA50EA22E4C0EEFFE5C005
:10095000EDFF7AC0E8F07BC0E9F07CC0EAF07DC032
:10096000EBF029CA02F0036A00EE16F0D950E9262E
:10097000DA50EA22EECF00F0EDCF01F0FE0E0026B5
:10098000FF0E0120016E78EC28F004C000F005C0D5
:1009900001F0026A036A0050E8270150E92302507F
:1009A000EA230350EB2329CA02F0036A00EE0EF09B
:1009B000D950E926DA50EA22EECF00F0EDCF01F06F
:1009C00012EC28F0026A036A0050E8270150E9237C
:1009D0000250EA230350EB23D9CFD0F0DACFD1F085
:1009E000E8C0ECF0E9C0EDF0EAC0EEF0EBC0EFF0EB
:1009F000DCC0F0F0DDC0F1F02B0EF26F0A0EF36FE9
:100A0000E0C0F4F0E1C0F5F00AEC1FF0006E00C0A9
:100A100002F0036A03500210D8B4000C0001DB514D
:100A2000D811D911DA11D8B4010CD890E435006E80
:100A3000E535016E2D0E0024E16E0C0E0120E26EF4
:100A400000EE16F0D051E926D151EA22E6CFEEFFB2
:100A5000E5CFEDFFD0C0E1FFD1C0E2FFE4C000F080
:100A6000E5C001F0E6C002F0E7C003F0002A000E86
:100A7000012200EE0EF0E150E926E250EA2200C029
:100A8000EEFF01C0EDFF7AC0E8F07BC0E9F07CC06A
:100A9000EAF07DC0EBF029CA02F0036A00EE16F01E
:100AA000E150E926E250EA22EECF00F0EDCF01F06E
:100AB000FE0E0026FF0E0120016E78EC28F004C027
:100AC00000F005C001F0026A036A0050E8270150F7
:100AD000E9230250EA230350EB2329CA02F0036AF8
:100AE00000EE0EF0E150E926E250EA22EECF00F0EF
:100AF000EDCF01F012EC28F0026A036A0050E827FB
:100B00000150E9230250EA230350EB23E8C0ECF044
:100B1000E9C0EDF0EAC0EEF0EBC0EFF0F06BF16B86
:100B20002C0EE025F26F0A0EE121F36FD8C0F4F02D
:100B3000D9C0F5F00AEC1FF0006E00C002F0036AA5
:100B400003500210D8B4000C010CC7007AC0C9F0E1
:100B50007BC0CAF07CC0CBF07DC0CCF0C7C0E1FF49
:100B6000C8C0E2FF29CA02F0036A00EE16F0E150A5
:100B7000E926E250EA22EECF00F0EDCF01F0FE0EC2
:100B80000026FF0E0120016E78EC28F004C000F072
:100B900005C001F0026A036A00010050C927015034
:100BA000CA230250CB230350CC2329CA02F0036A84
:100BB00000EE0EF0E150E926E250EA22EECF00F01E
:100BC000EDCF01F012EC28F0026A036A0050C92749
:100BD0000150CA230250CB230350CC23C9C0CFF00D
:100BE000CAC0D0F0CBC0D1F0CCC0D2F02B0ED36FA6
:100BF0000A0ED46F76EC1FF0006E00C002F0036A9C
:100C000003500210D8B4000C010CD96E15D0120E8E
:100C1000E8CF26FA010EE8CF27FA12D00A012653B0
:100C2000D8A40ED00A012753D8B4000C27CA00F06C
:100C30000028D8B4000C04D0D950E9E0010AEEE055
:100C400000018C0EC96F000ECA6F26CACBF027CAEE
:100C5000CCF0CD6BCE6B010ECF6F4ED92BCA26FADE
:100C60002CCA27FA010C00018C0EC96F000ECA6F46
:100C7000120ECB6FCC6BCD6BCE6B010ECF6F3CD910
:100C8000F66AF76A010ED96E11D0D950120AD8B49B
:100C90000CD0D950040D2B0EF324E96E0A0EF4206B
:100CA000EA6EEF50F626000EF722D92A230ED964F9
:100CB000ECD7F6CF00F0F7CF01F01200BA000F0129
:100CC000356B0001C26B0001C2519FDF0009D8B42F
:100CD0000ED1010E0001C26FF46A05D1F438E84666
:100CE000E00B020FF36EF3500AEE2BF0E926000E34
:100CF000EA22EF50D8B4F6D0F3500AEE2BF0E926F2
:100D0000000EEA22EF50800AD8B4ECD0F3501AEE6D
:100D10002CF0E126000EE222BCC0E9FFBDC0EAFFD4
:100D2000E7CFEFFFF3501AEE2DF0E126000EE2229E
:100D3000BEC0E9FFBFC0EAFFE7CFEFFFF3500AEE06
:100D400047F0E926000EEA22EF50006EF3500AEE5B
:100D500048F0E926000EEA22EF50036E00C002F0D0
:100D6000C0C0E9FFC1C0EAFF02C0EEFF03C0EDFF53
:100D7000020ED96ED92AD950130AD8B4010CD95011
:100D80000001BA25006E000EBB21016EFD0E00248D
:100D9000E96EFF0E0120EA6EEF50D8B411D0F35087
:100DA000D9CF00F0016A0026000E01222B0E00248C
:100DB000E96E0A0E0120EA6EEF50A00AD8B492D074
:100DC000D9500001BA25006E000EBB21016EFD0E48
:100DD0000024E96EFF0E0120EA6EEF50D8A411D076
:100DE000F350D9CF00F0016A0026000E01222B0E2D
:100DF0000024E96E0A0E0120EA6EEF50A00AD8A482
:100E000071D0D9500001BA25006E000EBB21016ED1
:100E1000FD0E0024E96EFF0E0120EA6EEF50D8A40B
:100E200011D0F350D9CF00F0016A0026000E012244
:100E30002B0E0024E96E0A0E0120EA6EEF50A00A84
:100E4000D8B4010CD9500001BA25006E000EBB21A8
:100E5000016EFD0E0024E96EFF0E0120EA6EEF50D8
:100E60003F0AD8A40FD0F350D9CF00F0016A002672
:100E7000000E01222B0E0024E96E0A0E0120EA6EFC
:100E80003F0EEF6ED9500001BA25006E000EBB2157
:100E9000016EFD0E0024E96EFF0E0120EA6EEF5098
:100EA0002A0AD8B4010CD950BA25006E000EBB2115
:100EB000016EFD0E0024E96EFF0E0120EA6EEF5078
:100EC000006EF350D9CF02F0036A0226000E03220F
:100ED0002B0E0224E96E0A0E0320EA6EEF50001872
:100EE000D8B448D7F42A070EF464F8D6ECD63E0EF0
:100EF000E8CF35FF000CC900CBC030FFCCC02FFFBE
:100F0000046A056A066A076A0001CB07CB29D8B4D0
:100F10001CD0CBC000F0016A0050000FF66E0150EB
:100F2000F76E100EF7220800F550016E006A000EF1
:100F300001BEFF0E026E036E005004260150052212
:100F40000250062203500722DFD70001CC51016E68
:100F5000006A000E01BEFF0E026E036E00500426F2
:100F6000015005220250062203500722CD510426CB
:100F7000010ED8B00526D8B00626D8B00726C9C0BD
:100F8000D0F0CAC0D1F004C0D2F005C0D3F006C082
:100F9000D4F007C0D5F0CEC0D6F0CFC0D7F021EC4A
:100FA00004F0010C006E046AD890FD0E01241AE3CF
:100FB000036AF00E011403E1040E036E013A026AA3
:100FC000D890032A0136FDE301320150005CD8B00D
:100FD000006E0236032EF8D704BE026C025004BE27
:100FE000006C1200013206E20132D8A0006AD890EB
:100FF0000032D8A0D89000C002F0006A0036ECD7CA
:1010000000151515151515151515151515151515A5
:1010100015151313131313131312121212121211A4
:1010200011111111111111111100FE81FE0000FEAC
:10103000C1FE0000FEE1FE0000FEF1FE0000FEF930
:10104000FE0000FEFDFE0000FEFFFE00181FC1F8BE
:101050000818423C817E322AE72A32E251E2649249
:10106000F5916561955C6202625CFA00F090FE3E6B
:101070003E363E3E384444282800FE7C3810103866
:101080007CFE0060FFF9DF600C1FFC1F0C88CCEEBB
:10109000CC882266EE6622387C7C7C382070A820C2
:1010A0003E0804FE04082040FE4020101054381072
:1010B0001038541010808894A28080A294888040B8
:1010C000707C7040041C7C1C0400000000000000C8
:1010D000BE0000000E000E0028FE28FE284854FE28
:1010E0005424462610C8C46C92AA44A000000A06E4
:1010F000000038448200008244380028107C102808
:1011000010107C101000A0600000101010101000D3
:10111000C0C0000040201008047CA2928A7C008499
:10112000FE800084C2A2928C42828A966230282479
:10113000FE204E8A8A8A7278949292600602E212A7
:101140000E6C9292926C0C9292523C00CCCC0000AD
:1011500000AC6C00001028448200282828282800B1
:10116000824428100402A2120C6492F2827CF824B9
:101170002224F8FE9292926C7C82828244FE8282C9
:101180004438FE92929282FE121212027C82929255
:10119000F4FE101010FE0082FE82004080827E026B
:1011A000FE10284482FE80808080FE041804FEFE2B
:1011B000081020FE7C8282827CFE1212120C7C823D
:1011C000A242BCFE1232528C4C929292640202FEF7
:1011D00002027E8080807E3E4080403EFE40304065
:1011E000FEC6281028C60E10E0100EC2A2928A86F3
:1011F00000FE8282000408102040008282FE000867
:10120000040204088080808080000204080040A856
:10121000A8A8F0FE908888707088888840708888B8
:1012200090FE70A8A8A83010FC12020410A8A8A86C
:1012300078FE100808F00090FA80004080887A005C
:1012400000FE2050880082FE8000F808F008F8F8C0
:10125000100808F07088888870F82828281008146A
:101260001418FCF81008081090A8A8A840087E8858
:10127000804078808040F8384080403878806080B6
:1012800078885020508818A0A0A07888C8A898888E
:1012900000106C82000000FE000000826C10000450
:1012A00002040804F0888488F00000000000FEFFBB
:1012B00033FFFEFFFFDBFF767EFFC3C3C3FFFFC329
:1012C000FF7EFFFFDBDBC3FFFF1B1B037EFFD3F7AC
:1012D00076FFFF18FFFF00FFFFFF0060E0C0FF7F09
:1012E000FFFF3CF7E3FFFFC0C0C0FF071C07FFFF85
:1012F0003F7EFCFF7EFFC3FF7EFFFF333F1E7EFF6E
:10130000E37FBEFFFF3BEFC6CEDFDBFB7303FFFFD8
:10131000FF037FFFC0FF7F3F7FE07F3FFFE038E0BC
:10132000FFC7FF38FFC70F1FF01F0FE3F3DBCFC767
:1013300000000000000000000000000000000000AD
:10134000000000000000000000000000000000009D
:10135000000000000000000000000000000000008D
:10136000000000000000000000000000000000007D
:10137000000000000000000000000000000000006D
:10138000000000000000000000000000000000005D
:10139000000000000000000000000000000000004D
:1013A000000000000000000000000000000000003D
:1013B000000000000000000000000000000000002D
:1013C000000000000000000000000000000000001D
:1013D000000000000000000000000000000000000D
:1013E00000000000000000000000000000000000FD
:1013F00000000000000000000000000000000000ED
:1014000000000000000000000000000000000000DC
:1014100000000000000000000000000000000000CC
:1014200000000000000000000000000000000000BC
:1014300000000000000000000000000000000000AC
:10144000000000000000000000000000000000009C
:10145000000000000000000000000000000000008C
:10146000000000000000000000000000000000007C
:10147000000000000000000000000000000000006C
:10148000000000000000000000000000000000005C
:10149000000000000000000000000000000000004C
:1014A000000000000000000000000000000000003C
:1014B000000000000000045450144400000000002C
:1014C0000000000000102210221010222022102004
:1014D00022202220402220224000000000000000A4
:1014E00000000000000000000000000000000000FC
:1014F00000000000000000000000000000000000EC
:10150000000000000000FE7BFF7BFEFE7AFE7AFEFC
:10151000FC78FC78FCF878F878F8F070F070F0E07F
:1015200060E060E0C040C040C000E020A0A0A0207B
:10153000A0A0A020A0A040800000000000000000AB
:10154000FCFC04048404F4946404F4A4E4047444EB
:10155000F4440404FCFC00000010F01000F05010F3
:1015600000E010100000000000000000000000007B
:101570008080808080800000000000000000FF006C
:1015800043300B005B6803784B320000FF002020E3
:10159000A8702000FEFFFEFEFEFEFEFEFECE86864A
:1015A00086CEFEFEFEFEFEFEFFFE0070887101F993
:1015B00000F901F90070897100F8002020A870205E
:1015C00000F8FEFF8F070303070707D8D8D8D8888D
:1015D00000001F101E101E101E101E101E101E10C8
:1015E0001F000000000000007F7F7F7F7F7F7F7FE4
:1015F0007F7F7F437F7F7F7F7F7F7F7F7F7F000035
:1016000000000000000000000000000000000000DA
:1016100000000000000003070F0F0E0E0F0F070061
:10162000000000000000D0D0D0D0D0D0D0D0D0D09A
:10163000D0D0D0D0D0D0D0D0D0D000E0B010F000FA
:10164000F010D05050700080E010F0000000E0B0CA
:1016500010F0000000000070D010D050D010D0501A
:10166000D010D0700000D0D0D0D0D0D0D0D0D0D03A
:10167000D0D0D0D0D0D0D0D0D0D0EEEEEEEEEEEEB6
:10168000EEEEEEEEEEEEEEEEEEEEEEEEEEEE000056
:10169000FF80FF007794A5BD837E003F202FE98463
:1016A000EC1800FF80FF000E0A0A0EE0BF80BFA00A
:1016B000BF80BFA0BF80BFE00000EEEEEEEEEEEE1A
:1016C000EEEEEEEEEEEEEEEEEEEEEEEEEEEEFDFD1C
:1016D000FDFDFDFDFDFDFDFDFDFDFDFDFDFDFDFD3A
:1016E000FDFD00007C50200C503C00000020403CE0
:1016F0000040007C4438007C54007C14680038446E
:10170000380038445434007C54007C540000FDFD03
:10171000FDFDFDFDFDFDFDFDFDFDFDFDFDFDFDFDF9
:10172000FD383A483A583A583A583A583A583A5896
:101730003A583A583A583A583A583A583A583A5819
:101740003A583A583A583A583A683A683A683A68C9
:101750003A683A783A883A683A783A983AA83AA889
:101760003AA83AA83AA83AD63BD63BD63BD63BA8AD
:101770003AD63BD63BD63BD63BD63BD63BD63BD6E2
:101780003BD63BD63BB83AC83AD83AD63BD63BD6FE
:101790003BD63BD63BD63BD63BE83AF83A083B181B
:1017A0003B283B383B483B583BD63BD63B683B78D5
:1017B0003B883B983BC63B7D6060606060606060DA
:1017C0006060606060607D007D53454C2E20443633
:1017D00034203A243F3F3F7D007D20313534312D88
:1017E00049494920284A44297D007D53454C2E20F3
:1017F000434152443A243020207D007D44495245E3
:1018000043544F52593A242020207D00726F6F7448
:10181000206469726563746F7279002573006A6071
:10182000606060606060606060606060606B0075F8
:1018300060606060606060606060606060606900FF
:1018400046696C653A2020253033642F2530336497
:101850000025633D2530326420543D25303264201C
:10186000533D25303264004452495645204E4F5472
:1018700020524541445900313534312D49494920E0
:1018800056005245434F5244204E4F54205052452B
:1018900053454E540046494C4520455849535453EE
:1018A00000494C4C4547414C2053595354454D2019
:1018B00054204F52205300494C4C4547414C205432
:1018C0005241434B20414E4420534543544F520014
:1018D0004449524543544F5259204552524F5200A9
:1018E00053594E544158204552524F520057524975
:1018F0005445204552524F520052454144204552D2
:10190000524F52004552524F5220554E4B4E4F5758
:101910004E0057524954452050524F54454354208D
:101920004F4E0046494C45204E4F54204F50454E97
:101930000057524954452046494C45204F50454E8A
:10194000004449534B2046554C4C004E4F204348D1
:10195000414E4E454C004F4B004E4F20424C4F43A2
:101960004B0046494C452054595045204D49534D54
:1019700041544348004449534B204944204D495366
:101980004D415443480046494C4520544F4F204C4C
:1019900041524745004F564552464C4F5720494EFD
:1019A000205245434F52440046494C45204E4F5427
:1019B00020464F554E440046494C45532053435210
:1019C000415443484544004E2F4100533A00433AA6
:1019D00000403A0053303A0043303A0040303A0079
:1019E00053656C656374696F6E206572722E004377
:1019F000617264206E6F7420737570702E00457272
:101A00003A256420622E626C2E000D0A0D0A2020F9
:101A10002D2D3D3D20313534312D49494920762544
:101A2000642E25642E25642C206279204A2E44657C
:101A3000726F676565203D3D2D2D000D0A4A3320EC
:101A400028426F6F746C6F61646572293A20444953
:101A50005341424C45442020286A756D70657220C0
:101A600072656D6F76656429000D0A4A322028443C
:101A700065766963652D494429203A2049443A2511
:101A8000642020202020286A756D706572207265A0
:101A90006D6F76656429000D0A4A332028426F6F06
:101AA000746C6F61646572293A204143544956450C
:101AB000202020286A756D70657220706C616365E6
:101AC0006429000D0A4A3220284465766963652D31
:101AD000494429203A2049443A25642020202020E6
:101AE00020286A756D70657220706C616365642969
:101AF00000240045723A766F6C74206572726F72C2
:101B0000210045723A434D443538206661696C21A5
:101B10000045723A696E69742E206661696C210015
:101B20004361726420646574656374656420002099
:101B300043415244204449524543544F5259200096
:101B4000496E69742E20636172643A20202000423D
:101B50004C4F434B5320465245452E2020202020F9
:0C1B600020202020202020202020000039
:101B6C009EB09E9064CFD8FF1000FAD7E9CF7EFFCD
:101B7C00EACF7DFFE1CF7CFFE2CF7BFFD9CF7AFFAD
:101B8C00DACF79FF0EC078FF0DC077FF0CC076FF5F
:101B9C000BC075FF0AC074FF09C073FF08C072FF49
:101BAC0007C071FF06C070FF05C06FFF04C06EFF59
:101BBC0003C06DFF02C06CFF01C06BFF00C06AFF69
:101BCC00F7CF69FFF6CF68FFF5CF67FFF4CF66FF5D
:101BDC00F3CF65FFF2A203D0F29201EC25F0F2A450
:101BEC0031D0D59EF2942CCFE8FF030AD8A420D094
:041BFC0011A804D058
:101C000011982ECFD6FF05D011882ECFE8FF0008FF
:101C1000D66ED7682ECF00F00004D8B411842ECF32
:101C2000E8FFFE0AD8B4119411A404D00F01010EEC
:101C30002E2B08D00F01010E2E0704D01178F60EBE
:101C4000D76ED66A11A802D0808201D08092D58E3C
:101C500065CFF3FF66CFF4FF67CFF5FF68CFF6FFE0
:101C600069CFF7FF6ACF00F06BCF01F06CCF02F0C5
:101C70006DCF03F06ECF04F06FCF05F070CF06F09C
:101C800071CF07F072CF08F073CF09F074CF0AF06C
:101C900075CF0BF076CF0CF077CF0DF078CF0EF03C
:101CA00079CFDAFF7ACFD9FF7BCFE2FF7CCFE1FF9C
:101CB0007DCFEAFF7ECFE9FF7FCFFAFF110081ECF5
:101CC00027F0080EE8CF34FF34CFE8FF38EC23F0DC
:101CD000119000010A0EDF6F1A0EE06F090EB86F47
:101CE000B96B070EB66FB76B060EB46FB56BB40E5B
:101CF000E8CFDDF0000EE8CFDEF09CEC28F000012C
:101D000082B010D0C30EDF6F1A0EE06F34CFB8F080
:101D1000B96BB80EE8CFDDF0000EE8CFDEF09CEC3A
:101D200028F00FD0690EDF6F1A0EE06F34CFB8F0D5
:101D3000B96BB80EE8CFDDF0000EE8CFDEF09CEC1A
:101D400028F0000182B207D0970EDF6F1A0EE06F05
:101D50009CEC28F006D03B0EDF6F1A0EE06F9CEC77
:101D600028F0118004EC25F032EC25F0010E000182
:101D7000C96F490EE1EC1CF00001080EBA6F070EA6
:101D8000BB6F01EC27F00F012D6B0001A96BA86B55
:101D9000C80E0001CE6FCF6BC2EC26F00001320EF0
:101DA000BA6F0F0EBB6F010EBC6FA8EC24F00001E0
:101DB000A56FA551D8A433D00F012D53D8A425D099
:101DC000010E1BEC27F01AEC25F075DB0009D8B4E6
:101DD0001CD0EEEC15F0030E0001C96F490EE1ECCA
:101DE0001CF000018A6B8B6B8AC0BAF08BC0BBF011
:101DF0000001BC6BBDEC14F00001C96BCA6BCB6B6E
:101E0000CC6BCD6B000EBAEC15F00001320EBA6F40
:101E10000F0EBB6F010EBC6FA8EC24F0C8D7C80E24
:101E20000001CE6FCF6BC2EC26F00001A551200A55
:101E3000D8B404D0A551400AD8A40BD00001A551B4
:101E4000200AD8A403D0010EA86FA2D7020E000169
:101E5000FBD70001A851D8A484D242EC23F098D734
:101E600042EC23F07CD242EC23F079D210EC1DF04E
:101E70008FD700013B0EBA6F0F0EBB6F010EBC6F08
:101E8000BD6B85DA320E0001BA6FBB6B01EC27F037
:101E90000001F10EBA6F1A0EBB6F3B0EBC6F0F0E36
:101EA000BD6F010EBE6FBF6B54EC26F001500010E9
:101EB0000001D8A486D03C0EBA6F0F0EBB6FB00ED7
:101EC000BC6F000EBD6F86DA006E00C002F0036AC0
:101ED00003500210D8B46CD00001B351B011B1114D
:101EE000B211D8A407D000018A6B8B6B010EE8CF2A
:101EF0002DFF63D0010EE8CF2DFF040E0001A96F66
:101F0000B0C08AF0B1C08BF0AC6BAD6BAE6BAF6B99
:101F10008AC000F08BC001F0026A036A000103501E
:101F2000AF5D08E10250AE5D05E10150AD5D02E13B
:101F30000050AC5DD8B034D00001AF51AC11AD1140
:101F4000AE11D8A408D08C0EBE6F000EBF6FC06B50
:101F50005CEC01F01ED000018C0EBE6F000EBF6F56
:101F6000010EC06F5CEC01F0006E00C002F0036A6D
:101F700003500210D8A40DD0020E0001C96F150E37
:101F8000E1EC1CF000018A6B8B6B010E0001A96F64
:101F900007D00001AC2B000EAD23AE23AF23B8D782
:101FA00000018C0EBA6F000EBB6F59EC03F0F0D637
:101FB00000018A518B11D8A402D0030E4CD0040E1C
:101FC0004AD0CB0EBA6F190EBB6F3B0EBC6F0F0E13
:101FD000BD6F020EBE6FBF6B54EC26F001500010B7
:101FE000D8B412D00001D40EBA6F190EBB6F3B0EDD
:101FF000BC6F0F0EBD6F030EBE6FBF6B54EC26F0AF
:1020000001500010D8A402D00A0E25D00001D10E34
:10201000BA6F190EBB6F3B0EBC6F0F0EBD6F020E79
:10202000BE6FBF6B54EC26F001500010D8B412D034
:102030000001DC0EBA6F190EBB6F3B0EBC6F0F0EAA
:10204000BD6F030EBE6FBF6B54EC26F00150001045
:10205000D8A403D0070E000163D00001CE0EBA6FE2
:10206000190EBB6F3B0EBC6F0F0EBD6F020EBE6F25
:10207000BF6B54EC26F0015000100001D8B412D010
:10208000D80EBA6F190EBB6F3B0EBC6F0F0EBD6F33
:10209000030EBE6FBF6B54EC26F001500010D8A4A5
:1020A00017D000013B0EBA6F0F0EBB6FA70EBC6FAF
:1020B000000EBD6FA60EBE6F000EBF6FAA0EC06FE2
:1020C000000EC16F5FEC06F00001A46F0C0E28D06B
:1020D00000018A518B1100013B0ED8A40DD0BA6FBC
:1020E0000F0EBB6F8C0EBC6F000EBD6F27EC1BF08C
:1020F0000001A46F060E14D0BA6F0F0EBB6FA70EAF
:10210000BC6F000EBD6FA60EBE6F000EBF6FAA0E95
:10211000C06F000EC16F5FEC06F00001A46F050EEA
:10212000A96F36D60F012D53D8B405D02DCFE8FFB7
:10213000020AD8A4EBD00001A851020AD8A403D007
:10214000010EA96FE3D0020E0001FBD742EC23F091
:10215000FBD085EC24F042EC23F0F6D042EC23F0E7
:10216000F3D0010E50DA8AC0BAF08BC0BBF0000188
:10217000BC6BBDEC14F05DEC17F0E6D0010E43DA59
:102180008AC0BAF08BC0BBF00001BC6BF6DB8AC022
:1021900000F08BC001F000500001BA6F0150BB6F1E
:1021A000BC6BBD6B31EC19F0CFD00001A851020A15
:1021B000D8A42FD0A405D8A421D0010E24DA020E71
:1021C0000001D76F000E4EEC25F000011B0EDF6FF3
:1021D000180EE06F3B0EB86F0F0EB96FB80EE8CF58
:1021E000DDF0000EE8CFDEF09CEC28F000018C0E54
:1021F000BA6F000EBB6FABEC1BF0A6D0020E000155
:10220000C96F3E0EE1EC1CF085EC24F042EC23F0AB
:102210009BD0020E0001C96F1C0EE1EC1CF0020EF7
:102220000001A96F91D00001A851020AD8A432D0B0
:10223000A405D8A424D0010EE6D9020E0001D76F60
:10224000000E4EEC25F000011B0EDF6F180EE06F44
:102250003B0EB86F0F0EB96FB80EE8CFDDF0000E71
:10226000E8CFDEF09CEC28F00001A651BA6FAAC0BE
:10227000BBF0ABC0BCF0A75151EC1CF065D0020E16
:102280000001C96F3E0EE1EC1CF085EC24F042EC3D
:1022900023F05AD00001A451020ED8A423D0B3D900
:1022A000020E0001D76F000E4EEC25F000011B0E50
:1022B000DF6F180EE06F3B0EB86F0F0EB96FB80EE0
:1022C000E8CFDDF0000EE8CFDEF09CEC28F0000156
:1022D000A651BA6FAAC0BBF0ABC0BCF0A751D3ECFB
:1022E0001CF032D00001C96F3F0EE1EC1CF042EC53
:1022F00023F02AD0050E87D927D0030E84D924D005
:10230000040E81D921D0060E7ED91ED00001A9511C
:1023100001E11CD7010A01E11CD7030A01E11ED724
:10232000010A01E11ED7070A01E128D7010A01E1EC
:102330007AD7030A01E139D7010ADCE00D0ADDE0B2
:10234000010ADEE0070ADFE0000E5DD921D542EC8C
:1023500023F0020E0001C96F1E0EE1EC1CF000011B
:1023600016D50001A5513F0A01E17AD5600A01E1C5
:102370007AD53F0A01E1D6D60F0A01E177D58F0A57
:1023800001E176D5100A01E174D5E1D7BA00119ABE
:1023900011960001BE6B0FD00001BC5148EC23F038
:1023A000006E0001BE51BA25E96E000EBB21EA6E37
:1023B00000C0EFFFBE2B11BA02D011A6EDD700016D
:1023C000BE51BA25E96E000EBB21EA6E000EEF6A1F
:1023D0001200BA00E16ABCC0D9FFBDC0DAFFD9CF94
:1023E000E9FFDACFEAFFEE6AEE6AEE6AED6A46D0FE
:1023F0000A0E046E056A066A076AD9CFE9FFDACFCA
:10240000EAFFEECF00F0EECF01F0EECF02F0EECF1C
:1024100003F0CFEC27F000C0DEFF01C0DEFF02C0FA
:10242000DEFF03C0DDFFDD52DD52E1500001BA25C1
:10243000E96E000EBB21EA6EEF50006E016AD00E0D
:102440000026FF0E0122026A036ADE500024046E99
:10245000DE500120056EDE500220066EDD500320A6
:10246000076EDD52DD5204C0DEFF05C0DEFF06C090
:10247000DEFF07C0DDFFDD52DD52E12AE150000141
:10248000BA25E96E000EBB21EA6EEF50006E300EE9
:10249000005CD8A00CD0E150BA25E96E000EBB213B
:1024A000EA6EEF50006E3A0E005CD8A0A1D7E15062
:1024B000D8B4000C010C0001D76B000E4EEC25F0D7
:1024C0000001200EDF6F1B0EE06F9CEC28F0020E67
:1024D0001BEC27F00001D76B000E4EEC25F000013D
:1024E000400EDF6F1B0EE06F9CEC28F0010E000128
:1024F000D76F000E4EEC25F02BD80009D8B422D0AF
:1025000024EC00F00009D8A40DD00001D76B000E18
:102510004EEC25F00001EF0EDF6F190EE06F9CEC22
:1025200028F0000C0001D76B0B0E4EEC25F00001DB
:10253000560EDF6F190EE06F9CEC28F0010EE8CF0D
:102540002DFF010C030E1BEC27F00F012D6B000C6F
:1025500025EC1EF00009D8A40DD025EC1EF00009D2
:102560000001D8A408D0110EDF6F1B0EE06F9CECA9
:1025700028F0000C0001360EBC6F0F0EBD6FC1ECD1
:102580001EF0006E00C002F0036A03500210D8A4CF
:1025900008D00001020EDF6F1B0EE06F9CEC28F0EC
:1025A000000C38CFE8FF3C0B3C0AD8B408D000013F
:1025B000F30EDF6F1A0EE06F9CEC28F0000C0001A8
:1025C000866B020E876F86C0BCF087C0BDF0FBEC47
:1025D0001EF0006E00C002F0036A03500210D8A47F
:1025E000010C0001FE0EDF6F190EE06F86C0BAF01D
:1025F00087C0BBF0BA0EE8CFDDF0000EE8CFDEF00A
:102600009CEC28F0000C0001BA6F030ED76F000E8F
:102610004EEC25F094D1200EAFEC27F0200EAFEC5D
:1026200027F08C0EAFEC27F08F0EAFEC27F0810E69
:10263000AFEC27F0840EAFEC27F0890EAFEC27F05B
:102640008E0EAFEC27F0870EAFEC27F02E0EAFEC1E
:1026500027F02E0EAFEC27F02E0EAFEC27F0200E59
:10266000AFEC27F069D1200EAFEC27F0200EAFECD5
:1026700027F0200EAFEC27F0930EAFEC27F0810E81
:10268000AFEC27F0960EAFEC27F0890EAFEC27F0F9
:102690008E0EAFEC27F0870EAFEC27F02E0EAFECCE
:1026A00027F02E0EAFEC27F02E0EAFEC27F0200E09
:1026B000AFEC27F041D1200EAFEC27F0200EAFECAD
:1026C00027F0840EAFEC27F0850EAFEC27F08C0ED0
:1026D000AFEC27F0850EAFEC27F0940EAFEC27F0AF
:1026E000890EAFEC27F08E0EAFEC27F0870EAFEC23
:1026F00027F02E0EAFEC27F02E0EAFEC27F02E0EAB
:10270000AFEC27F019D1200EAFEC27F0200EAFEC84
:1027100027F0920EAFEC27F0850EAFEC27F08E0E6F
:10272000AFEC27F0810EAFEC27F08D0EAFEC27F069
:10273000890EAFEC27F08E0EAFEC27F0870EAFECD2
:1027400027F02E0EAFEC27F02E0EAFEC27F02E0E5A
:10275000AFEC27F0F1D0200EAFEC27F0920EAFECEB
:1027600027F0850EAFEC27F0900EAFEC27F08C0E23
:10277000AFEC27F0810EAFEC27F0830EAFEC27F023
:10278000890EAFEC27F08E0EAFEC27F0870EAFEC82
:1027900027F02E0EAFEC27F02E0EAFEC27F02E0E0A
:1027A000AFEC27F0C9D0200EAFEC27F0200EAFEC35
:1027B00027F0830EAFEC27F08F0EAFEC27F0900ED2
:1027C000AFEC27F0990EAFEC27F0890EAFEC27F0B5
:1027D0008E0EAFEC27F0870EAFEC27F02E0EAFEC8D
:1027E00027F02E0EAFEC27F02E0EAFEC27F0200EC8
:1027F000AFEC27F0A1D0200EAFEC27F0860EAFECA7
:1028000027F08F0EAFEC27F0920EAFEC27F08D0E75
:10281000AFEC27F0810EAFEC27F0940EAFEC27F071
:10282000940EAFEC27F0890EAFEC27F08E0EAFECD4
:1028300027F0870EAFEC27F02E0EAFEC27F02E0E10
:10284000AFEC27F02E0EAFEF27F0200EAFEC27F005
:10285000200EAFEC27F0200EAFEC27F0920EAFEC7D
:1028600027F0850EAFEC27F0810EAFEC27F0840E39
:10287000AFEC27F0890EAFEC27F08E0EAFEC27F00F
:10288000870EAFEC27F02E0EAFEC27F02E0EAFEC3C
:1028900027F02E0EAFEC27F04FD0200EAFEC27F034
:1028A000200EAFEC27F0200EAFEC27F0570EAFEC68
:1028B00027F0920EAFEC27F0890EAFEC27F0940EC4
:1028C000AFEC27F0890EAFEC27F08E0EAFEC27F0BF
:1028D000870EAFEC27F02E0EAFEC27F02E0EAFECEC
:1028E00027F02E0EAFEC27F027D0200EAFEC27F00C
:1028F000200EAFEC27F0200EAFEC27F0200EAFEC4F
:1029000027F0200EAFEC27F0200EAFEC27F0200EC2
:10291000AFEC27F0200EAFEC27F0200EAFEC27F045
:10292000200EAFEC27F0200EAFEC27F0200EAFEC1E
:1029300027F0200EAFEC27F0200EAFEF27F00001BC
:10294000BA51010A01E167D6030A01E18CD6010AF6
:1029500001E1B1D6070A01E1D6D6010A01E1FBD6B1
:10296000030A01E120D7010A01E145D70F0A01E17D
:102970006CD7010A92E0B9D7BA000001BC05D8B4FF
:1029800081EC25F00001D76B000E4EEC25F0000124
:10299000400EDF6F180EE06F88C0BFF089C0C0F036
:1029A000BAC0BDF0BBC0BEF0BD0EE8CFDDF0000E7A
:1029B000E8CFDEF09CEC28F0010E0001D76F000E8E
:1029C0004EEC25F000015C0EDF6F1B0EE06F9CECFF
:1029D00028F0010E0001D76F000E4EEC25F000012B
:1029E000BB51BA11D8A408D00C0EDF6F180EE06FDF
:1029F0009CEC28F083EF25F08CC0E8FFAFEC27F0CB
:102A00008DC0E8FF200AD8A41ED08EC0E8FF200A9F
:102A1000D8A419D08FC0E8FF200AD8A414D090C041
:102A2000E8FF200AD8A40FD091C0E8FF200AD8A45C
:102A30000AD092C0E8FF200AD8A405D093C0E8FFCE
:102A4000200AD8B404D08DC0E8FFAFEC27F08EC0C8
:102A5000E8FF200AD8A419D08FC0E8FF200AD8A424
:102A600014D090C0E8FF200AD8A40FD091C0E8FF8E
:102A7000200AD8A40AD092C0E8FF200AD8A405D022
:102A800093C0E8FF200AD8B404D08EC0E8FFAFECB2
:102A900027F08FC0E8FF200AD8A414D090C0E8FF28
:102AA000200AD8A40FD091C0E8FF200AD8A40AD0E9
:102AB00092C0E8FF200AD8A405D093C0E8FF200AFE
:102AC000D8B404D08FC0E8FFAFEC27F090C0E8FF87
:102AD000200AD8A40FD091C0E8FF200AD8A40AD0B9
:102AE00092C0E8FF200AD8A405D093C0E8FF200ACE
:102AF000D8B404D090C0E8FFAFEC27F091C0E8FF55
:102B0000200AD8A40AD092C0E8FF200AD8A405D091
:102B100093C0E8FF200AD8B404D091C0E8FFAFEC1E
:102B200027F092C0E8FF200AD8A405D093C0E8FFA0
:102B3000200AD8B404D092C0E8FFAFEC27F093C0CD
:102B4000E8FF200AD8B404D093C0E8FFAFEC27F028
:102B50002E0EAFEC27F094C0E8FFAFEC27F095C045
:102B6000E8FFAFEC27F096C0E8FFAFEC27F083EF6B
:102B700025F0C9000001CE6F040ED76F000E4EEC99
:102B800025F00001CC51D76FCA5120EC26F0050E7C
:102B90000001D76F000E4EEC25F00001510EDF6FE3
:102BA000180EE06FC9C000F0016A00C0D5F001C086
:102BB000D6F0CEC000F0016A00C0D3F001C0D4F05E
:102BC00034CFD1F0D26B0D0ECF6FD06BCF0EE8CFDC
:102BD000DDF0000EE8CFDEF09CEF28F000018C0E57
:102BE000BE6F000EBF6FC06B5CEC01F0006E00C0EA
:102BF00002F0036A035002100001D8B421D0010E84
:102C0000886F896B00018C0EBE6F000EBF6F010EC6
:102C1000C06F5CEC01F0006E00C002F0036A03506C
:102C20000210D8B405D00001882B000E8923EAD702
:102C300000018C0EBE6F000EBF6FC06B5CEF01F029
:102C4000886B896B1200CCD811AE31D000018A514B
:102C50008B11D8B41AD08A51010A8B11D8B412D072
:102C600000018C0EBE6F000EBF6F020EC06F5CECD9
:102C700001F0006E00C002F0036A03500210D8B4E5
:102C800004D000018A07000E8B5B020EE8CF2DFFF7
:102C90008AC0BAF08BC0BBF0010E0001BC6F6DDEC4
:102CA00000015E0EBA6F010EBB6F01EC27F011AC94
:102CB0003BD088C002F089C003F08AC000F08BC00E
:102CC00001F00350015C02E10250005CD8B01AD060
:102CD00000018A518B11D8B412D000018C0EBE6F46
:102CE000000EBF6F010EC06F5CEC01F0006E00C003
:102CF00002F0036A03500210D8B404D000018A2BFA
:102D0000000E8B23020EE8CF2DFF8AC0BAF08BC0D5
:102D1000BBF0010E0001BC6F30DE00015E0EBA6F29
:102D2000010EBB6F01EC27F012A0120000019E51B2
:102D3000AB0ED8B49F19020ED8B4A019D8B4A151C3
:102D4000D8A42BD094C0E8FF440AD8A426D095C0BC
:102D5000E8FF360AD8A421D096C0E8FF340AD8A4E8
:102D60001CD000018C0EBA6F000EBB6F59EC03F043
:102D7000010EE8CF2DFF8AC0BAF08BC0BBF0000176
:102D8000BC6BFBDD00018A518B11D8A4CEEF1CF087
:102D9000030E0001C96FD0EF1CF0010E0001D76FC8
:102DA000000E4EEC25F081EC25F00001E00EDF6F07
:102DB000190EE06F9CEC28F083EC25F00001DC0E8E
:102DC000BA6F050EBB6F01EC27F08AC0BAF08BC05A
:102DD000BBF0010E0001BC6FD0D582A0080C090C1D
:102DE000046A056A066A076AC282C2B2FED7C45084
:102DF000016E006AC3500024026E000E0120036EB3
:102E0000000102C0A4F003C0A5F0000EA5BFFF0E94
:102E1000A66FA76F071808E10650A61905E105502F
:102E2000A51902E10450A419D8B40CD0A4C004F030
:102E3000A5C005F0A6C006F0A7C007F0C282C2A2D6
:102E4000D6D7FDD7119E1290119C00019A0EA42591
:102E5000A46FFC0EA521A56F6BEC28F00150800A31
:102E6000800F100ED8B4005CD8B002D0118E1200C2
:102E700000012F0EA425A46FFD0EA521A56F6BECFC
:102E800028F00150800A800F100ED8B4005CD8B032
:102E900002D0128012000001C10EA425A46FFD0E05
:102EA000A521A56F6BEC28F00150800A800F100E51
:102EB000D8B4005CD8A0118C1200010E0001C96FBB
:102EC000000EE1EC1CF0119685EC24F0010EB9EC3B
:102ED00023F0040EB9EC23F0010EB9EC23F0010E3F
:102EE000B9EC23F0000EB9EC23F0000EB9EC23F09E
:102EF000200EB9EC23F0120EB9EC23F0220EB9EC3F
:102F000023F000012F0EC96F1B0ECA6F38EC24F09E
:102F1000220EB9EC23F0000EB9EC23F0010EB9EC4F
:102F200023F0010EB9EC23F0000EB9EC23F0000EF3
:102F3000B9EC23F0200EB9EC23F0220EB9EC23F00B
:102F400000012F0EC96F180ECA6F38EC24F0220E44
:102F5000B9EC23F0000EB9EC23F0010EB9EC23F02C
:102F6000010EB9EC23F0000EB9EC23F0000EB9EC21
:102F700023F0200EB9EC23F0220EB9EC23F000016F
:102F8000D90EC96F170ECA6F38EC24F0220EB9ECB7
:102F900023F0000EB9EC23F0010EB9EC23F0010E82
:102FA000B9EC23F0000EB9EC23F0000EB9EC23F0DD
:102FB000200EB9EC23F0220EB9EC23F00001B70E7D
:102FC000C96F170ECA6F38EC24F0220EB9EC23F04B
:102FD000000EB9EC23F0010EB9EC23F0010EB9ECB0
:102FE00023F0000EB9EC23F0000EB9EC23F0200E14
:102FF000B9EC23F0220EB9EC23F00001FB0EC96FEF
:10300000170ECA6F38EC24F0220EB9EC23F0000E34
:10301000B9EC23F0010EB9EC23F0010EB9EC23F06A
:10302000000EB9EC23F0000EB9EC23F0200EB9EC41
:1030300023F0220EB9EC23F00001EA0EC96F170E3F
:10304000CA6F38EC24F0220EB9EC23F0000EB9EC74
:1030500023F0010EB9EC23F0010EB9EC23F0000EC1
:10306000B9EC23F0000EB9EC23F0200EB9EC23F0FC
:10307000220EB9EC23F00001C80EC96F170ECA6FFB
:1030800038EC24F0220EB9EC23F0000EB9EC23F05A
:10309000010EB9EC23F0010EB9EC23F0000EB9ECEF
:1030A00023F0000EB9EC23F0200EB9EC23F0220E31
:1030B000B9EC23F000011E0EC96F180ECA6F38EC70
:1030C00024F0220EB9EC23F0000EB9EC23F000013D
:1030D000BA6B8C0EBE6F000EBF6FC06B5CEC01F064
:1030E000006E00C002F0036A03500210D8B4A6D0EC
:1030F0000001BA2B00019E51AB0ED8B49F19020EED
:10310000D8B4A019D8B4A151D8A40FD094C0E8FF66
:10311000440AD8A40AD095C0E8FF360AD8A405D03E
:1031200096C0E8FF340AD8B40FD094C0E8FF500A24
:10313000D8A473D095C0E8FF520AD8A46ED096C028
:10314000E8FF470AD8A469D0010EB9EC23F0010EBC
:10315000B9EC23F00001BA51B9EC23F0026A010E78
:10316000036EBAC000F0016A45EC28F00450B9ECD7
:1031700023F00A0E0001BA6103D0200EB9EC23F04F
:10318000220EB9EC23F08CC0E8FFB9EC23F08DC01F
:10319000E8FFB9EC23F08EC0E8FFB9EC23F08FC054
:1031A000E8FFB9EC23F090C0E8FFB9EC23F091C040
:1031B000E8FFB9EC23F092C0E8FFB9EC23F093C02C
:1031C000E8FFB9EC23F02E0EB9EC23F094C0E8FF31
:1031D000B9EC23F095C0E8FFB9EC23F096C0E8FF06
:1031E000B9EC23F0220EB9EC23F0000EB9EC23F079
:1031F0000001C96BBA5188C000F089C001F0005CC1
:10320000CA6F0150D8A00104CB6F00EECCF088C08B
:10321000EEFF89C0EDFF000EADDC00018C0EBE6F2D
:10322000000EBF6F010EC06F5CEC01F0006E00C0BD
:1032300002F0036A03500210D8A45AD700018C0E82
:10324000BE6F000EBF6FC06B5CEC01F0000EB9ECFE
:1032500023F01186000EB9EC23F096EC24F098D5FB
:10326000BA00010E0001C96F000EABDB119685ECB0
:1032700024F0010EB9EC23F0040EB9EC23F00001A8
:103280008C0EC96F000ECA6F120ECB6FCC6B900EF6
:10329000CD6F190ECE6FCF6B7CEC07F0010E0001E5
:1032A000C76FC86BC96B010ECA6FCB6BCC6BCD6B94
:1032B000120E60DC010EB9EC23F0010EB9EC23F024
:1032C0000001BA51B9EC23F00001BB51B9EC23F075
:1032D000120EB9EC23F0220EB9EC23F00001C16B01
:1032E0000001C1510AEE2BF0E926000EEA22EF5050
:1032F000B9EC23F00001C12B0F0EC165F1D7220EEE
:10330000B9EC23F0200EB9EC23F03DCAE8FFB9EC8C
:1033100023F03ECAE8FFB9EC23F0200EB9EC23F00D
:1033200040CAE8FFB9EC23F041CAE8FFB9EC23F04A
:10333000000EB9EC23F00001BE6B0001BE5105EC9C
:1033400006F00009D8B45BD10001C74BC82B2FCFC2
:10335000C9F0C7C0CAF0C8C0CBF0CC6BCD6B30CFC2
:10336000E8FF08DC010E0001BE6FBF6B43D1000116
:10337000BF39E846E00B020FC26FC2510AEE2BF0D4
:10338000E926000EEA22EF50D8B432D1010EB9EC92
:1033900023F0010EB9EC23F00001C2510AEE47F010
:1033A000E926000EEA22EF50B9EC23F00001C251E9
:1033B0000AEE48F0E926000EEA22EF50B9EC23F0BD
:1033C0000001C2510AEE47F0E926000EEA22EF5052
:1033D000006EC2510AEE48F0E926000EEA22EF50D4
:1033E000C66F00C0C5F0000EC65D0A0ED8B4C55D3C
:1033F000D8B003D0200EB9EC23F00001000EC65D5A
:10340000640ED8B4C55DD8B003D0200EB9EC23F05B
:103410000001030EC65DE80ED8B4C55DD8B003D078
:10342000200EB9EC23F0220EB9EC23F00001C06BA2
:10343000030EC16F0001C251C1C000F0016A002635
:10344000000E01222B0E0024E96E0A0E0120EA6E06
:10345000EF50A00AD8B411D0C251C1C000F0016A27
:103460000026000E01222B0E0024E96E0A0E012018
:10347000EA6EEF50200AD8A408D00001C02B1AD061
:10348000200EB9EC23F00001C0070001C051D8A400
:10349000F7D70001C251C1C000F0016A0026000E3A
:1034A00001222B0E0024E96E0A0E0120EA6EEF5075
:1034B000B9EC23F00001C12B120EC165BBD7220E5F
:1034C000B9EC23F00001C051D8B406D0200EB9ECFD
:1034D00023F00001C007F6D70001C2510AEE2BF01D
:1034E000E926000EEA22EF50006E800E005CD8A0A4
:1034F00004D0200EB9EC23F036D02A0EB9EC23F01C
:1035000032D0440EB9EC23F0450EB9EC23F04C0E4A
:10351000B9EC23F04DD0530EB9EC23F0450EB9ECC5
:1035200023F0510EB9EC23F043D0500EB9EC23F048
:10353000520EB9EC23F0470EB9EC23F039D0550EFA
:10354000B9EC23F0530EB9EC23F0520EB9EC23F092
:103550002FD0520EB9EC23F0450EB9EC23F04C0EEF
:10356000B9EC23F025D00001C2510AEE2BF0E92678
:10357000000EEA22EF50006E070E001600C002F0A7
:10358000036A0BD00250BDE0010AC5E0030ACDE09A
:10359000010AD5E0070ADDE002D00350F3E0550E42
:1035A000B9EC23F04E0EB9EC23F04B0EB9EC23F03E
:1035B0000001C2510AEE2BF0E926000EEA22EF507C
:1035C000006EC00E005CD8A004D03C0EB9EC23F015
:1035D00003D0200EB9EC23F0200EB9EC23F0200E1E
:1035E000B9EC23F0200EB9EC23F0000EB9EC23F077
:1035F0000001BF2B070E0001BF65B9D69ED6010E94
:10360000B9EC23F0010EB9EC23F033EC06F000C066
:10361000C3F001C0C4F00001C351B9EC23F00001B4
:10362000C451B9EC23F000014F0EC96F1B0ECA6FD5
:1036300038EC24F0000EB9EC23F0000EB9EC23F0C6
:103640001186000EB9EC23F096EC24F0A7D1BCC093
:10365000BEF0BDC0BFF00001C06B5CEC01F0006EBD
:1036600000C002F0036A03500210D8B4000CD968FD
:10367000D92ABCC0E1FFBDC0E2FFD950080AD8A4D6
:103680001ED000EE08F0E150E926E250EA22EF50A9
:10369000500AD8A414D000EE09F0E150E926E25017
:1036A000EA22EF50520AD8A40AD000EE0AF0E15004
:1036B000E926E250EA22EF50470AD8B4010C000193
:1036C000BA51D924E96E000ED9BEFF0EBB21EA6EB5
:1036D000EF50D8B436D00001BA51D924E96E000EAB
:1036E000D9BEFF0EBB21EA6EEF503F0AD8A408D026
:1036F000D950E124E96E000EE220EA6E3F0EEF6E33
:103700000001BA51D924E96E000ED9BEFF0EBB21CB
:10371000EA6EEF502A0AD8B4010CBA51D924E96EE6
:10372000000ED9BEFF0EBB21EA6EEF50006ED950DD
:10373000E124E96E000EE220EA6EEF500018D8B4E2
:1037400097D7BCC0BEF0BDC0BFF0010E0001C06F76
:103750005CEC01F084D7010E0001C96F000E31D975
:10376000119685EC24F0BAC0E1FFBBC0E2FF00EE89
:1037700012F0E150E926E250EA22EECFC3F0EECF9C
:10378000C4F0EECFC5F0EECFC6F00001BF6BC06B4A
:10379000BC6BFE0E046E056A066A076AC3C000F0C1
:1037A000C4C001F0C5C002F0C6C003F026EC27F08B
:1037B00000C0C1F001C0C2F0C1C0BDF0C2C0BEF0C7
:1037C000FE0E046E056A066A076AC3C000F0C4C034
:1037D00001F0C5C002F0C6C003F026EC27F0075088
:1037E000041005100610D8B402D0C14BC22B000142
:1037F000C107D8A0C207E1CFC7F0E2CFC8F0A6EC5E
:1038000005F00001C651C311C411C511D8B444D08C
:103810000001C305C411C511C611D8B411860AEE42
:103820002BF0BF51E926C051EA22EF50B9EC23F04A
:103830000001C307000EC45BC55BC65BBC2BBF4B5E
:10384000C02BC051020ABF11D8A40FD0BAC0C7F014
:10385000BBC0C8F098EC03F0BAC0C7F0BBC0C8F05A
:10386000A6EC05F00001BF6BC06B0001BC51FE0A65
:10387000D8A4C7D7C107D8A0C207C96BC1C0CAF0B6
:10388000C2C0CBF0BDC0CCF0BEC0CDF0000EBAECD3
:1038900015F00001BC6BB5D796EC24F0C8EF16F01C
:1038A000BA000001BD6FBBC0C3F0BCC0C4F0010EC4
:1038B000C96F000E86D8119685EC24F00001BA512C
:1038C000C96FC3C0CAF0C4C0CBF0BBC0CCF0BCC091
:1038D000CDF0BD51BAEC15F00001BD51C16FC26B06
:1038E000BA51BF6FC06B8C0EC96F000ECA6FBD514D
:1038F000CB6FBA51CC6FCD6BCE6B010ECF6F7CEC22
:1039000007F02BCABDF02CCABAF00001C307D8A03B
:10391000C407BD51D8B412D0020EBE6F0001BE5113
:103920000AEE2BF0E926000EEA22EF50B9EC23F064
:103930000001BE2BBE51D8B4C1D7F0D70001BF5192
:10394000C96FC3C0CAF0C4C0CBF0BBC0CCF0BCC010
:10395000CDF0C151BAEC15F0020E0001BE6F0001AE
:10396000BA51BE5DD8B00DD00001BE510AEE2BF0A9
:10397000E926000EEA22EF50B9EC23F00001BE2B3D
:10398000EED711860001BA510AEE2BF0E926000E9F
:10399000EA22EF50B9EC23F096EC24F00001C96B59
:1039A000000E0FD0BA00BBC0F3FFBCC0F4FF010E85
:1039B0000001C96F000E05D80A0E1BEC27F0EED7E8
:1039C000C900D96ED950D8B421D035CFE8FF490A03
:1039D000D8A4D9CF35FF1AD0D59E80921200D59E9B
:1039E00080821200020EE8CF2CFF1198D768D668AB
:1039F000D58E1200030EE8CF2CFF11941198D768D2
:103A0000D668D58E1200D59E809212000001C95151
:103A1000E3E0010AE4E0030AE5E0010AEBE0F3D7A2
:103A20001196808285EC24F035CFE8FF6DEC24F010
:103A30002C0EB9EC23F0D7D00001560EC96F190E29
:103A4000CA6F38EC24F0E3D00001B70EC96F190E2D
:103A5000CA6F38EC24F0DBD00001C70EC96F190E15
:103A6000CA6F38EC24F0D3D00001F90EC96F180EDC
:103A7000CA6F38EC24F0CBD00001ED0EC96F180EE0
:103A8000CA6F38EC24F0C3D00001120EC96F190EB2
:103A9000CA6F38EC24F0BBD00001750EC96F190E47
:103AA000CA6F38EC24F0B3D00001E00EC96F180ED5
:103AB000CA6F38EC24F0ABD00001820EC96F180E2B
:103AC000CA6F38EC24F0A3D00001950EC96F190E0F
:103AD000CA6F38EC24F09BD00001860EC96F190E16
:103AE000CA6F38EC24F093D00001310EC96F190E63
:103AF000CA6F38EC24F08BD00001230EC96F190E69
:103B0000CA6F38EC24F083D00001A80EC96F190EDB
:103B1000CA6F38EC24F07BD00001950EC96F180EE7
:103B2000CA6F38EC24F073D00001620EC96F190E11
:103B3000CA6F38EC24F06BD00001590EC96F190E12
:103B4000CA6F38EC24F063D00001B70EC96F180EAD
:103B5000CA6F38EC24F05BD00001A10EC96F180EBB
:103B6000CA6F38EC24F053D000014B0EC96F190E08
:103B7000CA6F38EC24F04BD00001D00EC96F180E7C
:103B8000CA6F38EC24F043D00001410EC96F190E02
:103B9000CA6F38EC24F03BD00001770EC96F180EC5
:103BA000CA6F38EC24F0060E6DEC24F02E0EB9EC42
:103BB00023F0070E6DEC24F02E0EB9EC23F0090E65
:103BC0006DEC24F024D00001670EC96F180ECA6F87
:103BD00038EC24F01CD00001040EC96F190ECA6F16
:103BE00038EC24F014D035CFE8FF000FF4E6B50F21
:103BF000F2E74B0F020D210EF324F66E170EF420A0
:103C0000F76E0900F5500900F5CFFAFFF96E320E94
:103C10000001BA6FBB6B01EC27F02C0EB9EC23F05E
:103C200030CFE8FF6DEC24F02C0EB9EC23F02FCF51
:103C3000E8FF6DEC24F011860D0EB9EC23F096EC44
:103C400024F080920F01356B1200C696C694C6828E
:103C5000C69082840001BC6BBD6BFF0ECAEC27F0DE
:103C60000001BC4BBD2B000EBD5D0A0ED8B4BC5D7F
:103C7000D8A0F3D78294F36AF46AF34AF42AC30E05
:103C8000F45C500ED8B4F35CD8A0F7D70001F66B03
:103C9000F76BF86BF96B400E09DA21CA00F00004EB
:103CA000D8A4000C0001F66BF76BF86BF96B770E7C
:103CB000FDD921CAE8FF050AD8A422D00001746BFF
:103CC000756B010EE8CF21FA0A012153D8B413D045
:103CD0000001F66BF76BF86BF96B410EE7D9000149
:103CE0007551270A100ED8B47419D8B4000C742B6F
:103CF000000E7523E9D7C696C694C692C680010CFD
:103D00000001746B756B010EE8CF21FA0A01215393
:103D1000D8B41AD00001F66BF76BF86BF96B690E2B
:103D2000C5D90001F66BF76BF86BF96B770EBED94E
:103D300000017551270A100ED8B47419D8B4000CBC
:103D4000742B000E7523E2D7C696C694C692C68021
:103D5000010CA4000001A46BA56BA66BA76B4D0E14
:103D6000B7D9A4C0E1FFA5C0E2FF00EE01F0E15029
:103D7000E926E250EA2221CAEFFF22CAE7FF010C3E
:103D8000BC000001746B756B010EE8CF21FA0A01CB
:103D90002153D8B410D00001BE6BBF6BC06BC16B98
:103DA0007A0EADD90001741D7511D8B4000C742BB6
:103DB000000E7523ECD7BCC0E1FFBDC0E2FF00EEF2
:103DC00003F0E150E926E250EA2222CAEFFF00EEBA
:103DD00002F0E150E926E250EA2223CAEFFF00EEAA
:103DE00001F0E150E926E250EA2224CAEFFF25CA99
:103DF000E7FF010CBC000001F66BF76BBCC0F8F0EC
:103E0000BDC0F9F0500E52D90A012153D8A4000CBC
:103E1000010CEC000001090ED890EC37ED37EE37BD
:103E2000EF37E82EF9D7EEC0F6FFEFC0F7FFECC092
:103E3000F3FFEDC0F4FFF6CFF6F0F7CFF7F0F3CFD6
:103E4000F8F0F4CFF9F0510E31D90A012153D8A47A
:103E5000000C0001746B756BFF0ECAEC27F0FE0AB4
:103E6000D8B412D0000174C000F075C001F0002871
:103E7000746F02E10128756F030E015CE80ED8B47F
:103E8000005CD8B0000CE8D7F2C0E1FFF3C0E2FF5D
:103E9000006A016A026A036AC968C7A0FED7000106
:103EA000F151F011D8A403D0C9CFE6FF06D0C9CF95
:103EB000E7FF0001F007D8A0F107002A000E012259
:103EC00002220322035C08E1000E025C05E1020EFF
:103ED000015C02E1000E005CD8A0DED7FF0ECAEC48
:103EE00027F0FF0ECAEC27F0010CCF000001090EED
:103EF000D890CF37D037D137D237E82EF9D7D1C0C5
:103F0000F3FFD2C0F4FFCFC0F6FFD0C0F7FFF3CF6E
:103F1000F6F0F4CFF7F0F6CFF8F0F7CFF9F0510E56
:103F2000C5D80A012153D8A4000C0001746B756B2D
:103F3000FF0ECAEC27F0FE0AD8B412D0000174C0FC
:103F400000F075C001F00028746F02E10128756F60
:103F5000030E015CE80ED8B4005CD8B0000CE8D7C2
:103F6000D3C0E1FFD4C0E2FFD96AC968C7A0FED7B9
:103F7000C9CFE6FFD92EF9D7C968C7A0FED7C9CFE8
:103F8000E6FFD92EF9D7FF0ECAEC27F0FF0ECAECD8
:103F900027F0010CA4000001090ED890A437A53722
:103FA000A637A737E82EF9D7A6C0F6FFA7C0F7FFB8
:103FB000A4C0F3FFA5C0F4FFF6CFF6F0F7CFF7F0FB
:103FC000F3CFF8F0F4CFF9F0580E70D80A0121536E
:103FD000D8A4000CFF0ECAEC27F0FF0ECAEC27F0A5
:103FE000FE0ECAEC27F00001A56BA66B0001A551DF
:103FF000A825E96EA651A921EA6EEF50CAEC27F078
:104000000001A54BA62B020EA65D000ED8B4A55D3F
:10401000D8A0ECD7FF0ECAEC27F0FF0ECAEC27F0B1
:10402000FF0ECAEC27F00001A46FFF0ECAEC27F0C8
:10403000006E0028D8B4010CF8D7FB000001FF6F18
:104040000A01206BFF0ECAEC27F00001FF51CAECF9
:1040500027F00001FF5178D80001FC51CAEC27F08D
:104060000001FC5171D80001FB51CAEC27F000019E
:10407000FB516AD80001FE51CAEC27F00001FE5145
:1040800063D80001FD51CAEC27F00001FD515CD856
:104090000AEE20F0D890EF360A01202B20CAE8FF64
:1040A000CAEC27F0FF0ECAEF27F0F6000001FA6F06
:1040B000F6C0FBF0F7C0FCF0F8C0FDF0F9C0FEF070
:1040C000BDDFFF0ECAEC27F0E8CF21FA1200A400F2
:1040D0000001A46FA4C0FBF0A5C0FCF0A6C0FDF0D9
:1040E000A7C0FEF0ABDFFF0ECAEC27F0E8CF21FA45
:1040F000FF0ECAEC27F0E8CF22FA1200BE00000142
:10410000C26FBEC0FBF0BFC0FCF0C0C0FDF0C1C0BC
:10411000FEF094DFFF0ECAEC27F0E8CF21FAFF0E85
:10412000CAEC27F0E8CF22FAFF0ECAEC27F0E8CF5E
:1041300023FAFF0ECAEC27F0E8CF24FAFF0ECAECF0
:1041400027F0E8CF25FA1200D96E080EE16E0AEECC
:1041500020F0D890EF360A01D9AE02D0090E201B0C
:1041600020AF03D00A01090E201BD890D936E12ECA
:10417000EED71200F200F2C0F6FFF3C0F7FF0F0E09
:10418000F76403D00800F55005D0F6CFE9FFF7CF6C
:10419000EAFFEF501200DD000001E86BE96BDDC0C3
:1041A000E1FFDEC0E2FF0001E151F26FE251F36F87
:1041B000E14BE22BE0DF0001E76FE751D8B432D2E8
:1041C0000001E751250AD8B404D0E751E36F38DA8B
:1041D000EAD70001E469E66BE56BE1D10001E0514B
:1041E000DF11D8B406D0DFC0E9FFE0C0EAFF000E5F
:1041F000EF6AE8C000F0E9C001F01200E1CFE9FF8A
:10420000E2CFEAFF020EE126000EE222EF500001AB
:1042100002D20001E58DC3D10001E58FC0D10001BC
:10422000E52B0A0E04D0100E01D0080E0001E46F39
:104230000001E5AF09D0E6CFEAF0E6CFEBF0E6CF3C
:10424000ECF0E6CFEDF018D0E1CFE9FFE2CFEAFFE6
:10425000020EE126000EE222EECF00F0EDCF01F0DB
:1042600001BEFF0E026E036E00C0EAF001C0EBF06B
:1042700002C0ECF003C0EDF00001E5A124D0EDAFE9
:104280001DD0EAC000F0EBC001F0ECC002F0EDC0C0
:1042900003F0001E011E021E031E002AD8B4012ACC
:1042A000D8B4022AD8B4032A00C0EAF001C0EBF067
:1042B00002C0ECF003C0EDF0E6070FD00001E5917D
:1042C000E5AD0BD0F9D70001E5BF05D0EA51EB51C0
:1042D000EB6FEC6BED6B0001E591E4C004F0056A57
:1042E000066A076AEAC000F0EBC001F0ECC002F019
:1042F000EDC003F026EC27F004500001E76FE4C0A6
:1043000004F0056A066A076AEA0EE96E000EEA6EB4
:10431000BBEC28F0010EEE6FEF6BF06BF16B000160
:10432000F151ED5D08E1F051EC5D05E1EF51EB5D20
:1043300002E1EE51EA5DD8A00ED0E4C004F0056AB7
:10434000066A076AEE0EE96E000EEA6EA7EC28F028
:104350000001E607E4D70001E5A905D00BD0200E47
:104360000001E36F6DD90001E607E651800A7F0F77
:10437000D8B0F5D70001E5A104D02D0EE36F60D9C8
:1043800006D00001E5AD03D02B0EE36F59D9000133
:10439000E5B905D034D0300E0001E36F51D90001EA
:1043A000E607E651800A7F0FD8A029D0F4D7EEC0E7
:1043B00004F0EFC005F0F0C006F0F1C007F0EAC06D
:1043C00000F0EBC001F0ECC002F0EDC003F026EC11
:1043D00027F0E4C004F0056A066A076A26EC27F0B5
:1043E00004500001E66FE651800A760FD8A002D093
:1043F000070EE6270001E651300FE36F21D9E4C034
:1044000004F0056A066A076AEE0EE96E000EEA6EAF
:10441000BBEC28F00350001001100210D8A4C7D73D
:10442000090E0001E76502D0070EE7270001E751FA
:10443000300FE36F05D9B7D60001E651800A7E0F31
:10444000D8A006D0200E0001E36FFAD8E607F4D713
:10445000E1CFE9FFE2CFEAFF020EE126000EE22201
:10446000EF500001E76FE751E36FEAD89CD6E1CF48
:10447000E9FFE2CFEAFF020EE126000EE222EECFD4
:1044800000F0EDCF01F000C076F001C077F0000140
:10449000E76B76C000F077C001F00001E75100241F
:1044A000026E000E0120036E02C0F6FF03C0F7FF8C
:1044B0000F0EF76403D00800F55005D0F6CFE9FFE2
:1044C000F7CFEAFFEF500009D8B403D00001E72B83
:1044D000E0D70001E451E76102D0E751E46F000149
:1044E000E451E6BF1ED0FF0AE625D8A01AD0200E60
:1044F0000001E36FA5D8E607F2D7000176C000F00F
:1045000077C001F00028766F02E10128776F00C0C4
:10451000F2F001C0F3F02FDE0001E76FE751E36F27
:104520008FD80001E407E429D8B43DD6E6D7E1C02E
:10453000F2F0E2C0F3F01FDE2A0AD8A40ED0E1CFD9
:10454000E9FFE2CFEAFF020EE126000EE222EF5081
:104550000001E46FE14BE22B22D00001E151F26F48
:10456000E251F36FE14BE22B06DED00F0001E46F66
:10457000E1C0F2F0E2C0F3F0FEDD0001E76F2F0EC4
:10458000E7650DD03A0EE7610AD0E4510A0DE75114
:10459000F324D00FDED70001E5B530D0E589000166
:1045A000E151F26FE251F36FE14BE22BE4DD0001E8
:1045B000E76FE75101E112D62A0A01E11FD6010A8D
:1045C00001E127D6050AB3E01E0AE5E0680A01E129
:1045D0002AD63B0A01E130D7070A01E120D6080AB2
:1045E00001E11AD6030A01E120D61C0A01E13FD7F6
:1045F000060A01E11DD60D0A01E115D62F0E0001B4
:10460000E7650BD03A0EE76108D0E585E6510A0D63
:10461000E751F324D00FE66FC2D70001E751E36FF3
:104620000FD8C1D50001E051DF11D8B406D0DFC0EA
:10463000E9FFE0C0EAFF000EEF6A0001E72B13D0AC
:10464000E84BE92BE051DF11D8B409D0DFC0E9FF16
:10465000E0C0EAFFE3C0EFFFDF4BE02B12000001F8
:10466000E351AFEF27F0E8C000F0E9C001F012001D
:104670000001BA6FB6D9BCD9C1D91196119ABAC086
:104680002BFF1200AED9B4D9B9D981B01200FDD731
:104690000001BF6F1196119AC16B080EC06F80A404
:1046A000FED7ACD90001880EC26F130EC36F000E87
:1046B000C46FC56F000180A44BD0C207000EC35B5E
:1046C000C45BC55BC551C211C311C411D8A4F2D7D4
:1046D000118697D9460E0001CE6FCF6BC2EC26F043
:1046E0008DD9E8D70001D890C133C007880E006E7D
:1046F000130E016E000E026E036E80A4FED700063C
:10470000000E015A025A035A035000100110021001
:10471000D8A402D0118A000C80A603D0800E00011C
:10472000C127880E006E130E016E000E026E036E1E
:1047300080B4FED70006000E015A025A035A0350F5
:10474000001001100210D8A402D0118A000C000140
:10475000C051D8A4C7D70001BF51D8A406D0E20EDB
:10476000CE6F040ECF6FC2EC26F04BD90001C151C1
:1047700012000001CC6F080ECD6F119A39D980A6B6
:10478000FED711A632D0C80E0001CE6FCF6BC2EC9F
:1047900026F0880E006E130E016E000E026E036E80
:1047A00080B6FED70006000E015A025A035A035083
:1047B000001001100210D8A402D0118A000C880E3B
:1047C000006E130E016E000E026E036E80A6FED701
:1047D0000006000E015A025A035A0350001001103D
:1047E0000210D8A402D0118A000C05D9500E000185
:1047F000CE6FCF6BC2EC26F00001CD51D8B418D0EB
:10480000FAD8500E0001CE6FCF6BC2EC26F000013B
:10481000CD07CCA102D0F2D801D0F3D8E9D800015D
:10482000D890CC33500ECE6FCF6BC2EC26F0E4D7CD
:10483000E2D8E4D8880E006E130E016E000E026EF0
:10484000036E80B6FED70006000E015A025A035AC4
:104850000350001001100210D8A402D0118A000CDD
:10486000640E0001CE6FCF6BC2EC26F0010CC900C4
:104870000001CB6B0001CB51C925006E000ECA218F
:10488000016E00C0F6FF01C0F7FF0F0EF76403D002
:104890000800F55005D0F6CFE9FFF7CFEAFFEF505B
:1048A0000009D8B412000001CB51C925006E000EDA
:1048B000CA21016E00C0F6FF01C0F7FF0F0EF764BA
:1048C00003D00800F55005D0F6CFE9FFF7CFEAFF97
:1048D000EF504FDF0001CB2BCDD7D96E0A0E016E02
:1048E000D950D2EC07F0300F0001BB6FD950BA6F2E
:1048F000BB513FDF0A0E016E0001BA51D2EC07F046
:104900000050300FBB6FBB5134D780A4FED776D890
:104910003C0E0001CE6FCF6BC2EC26F06CD83C0E83
:104920000001CE6FCF6BC2EC26F0010C6AD83C0EB2
:104930000001CE6FCF6BC2EC26F05AD83C0E0001BE
:10494000CE6FCF6BC2EC26F080A4010CFDD7BA006D
:10495000C80E0001CE6FCF6BC2EC26F081A002D052
:104960004DD8000C4ED80001BC5192DEBAC0E9FF10
:10497000BBC0EAFFEF6EBAC0E1FFBBC0E2FFE75089
:104980000F0BD96E11AA81B0000CE750006E2BCF2F
:10499000E8FF20090018D8B4200CE7503F0AD8B42B
:1049A0003F0CE750006E2BCFE8FF40090018D8B449
:1049B000400CE7505F0AD8B45F0CE750F00BF00AE8
:1049C000D8B4F00CE750F00BE00AD8B4E00CE75094
:1049D000F00B600AD8A4000CD9500F0AD8B46F0CA1
:1049E000600C8180938012009350936E819012002E
:1049F0008084928412009294809412008086928621
:104A00001200929680961200819C819E818A8198E4
:104A10008194320EDDEC26F08184819A210E48D8F3
:104A2000BB0E46D8060E44D8130E42D8200E40D8EE
:104A30000C0E3ED00001D76B000E30D80001F80EEE
:104A4000BA6F010EBB6F0001BA51006EBB51016E0F
:104A5000BA07000EBB5B01500010D8B41200000E64
:104A60004DD8F1D70001D76B000E18D80001BA6BF2
:104A7000BB6B0001BB05F80ED8B4BA19D8B412004C
:104A8000BA4BBB2BBA51290FF66EBB51F76E150E00
:104A9000F7220800F55032D8ECD7D7000001D86FC4
:104AA000D851060DF350800F03D80001D751400FA5
:104AB000E96E8198E950E16E080ED96ED950D8B4EC
:104AC0001200819C010EE8CF28FA0A0100F000F0E4
:104AD000282F66EF25F0D906E1AE02D0818E01D0F5
:104AE000819E818C010EE8CF28FA0A0100F000F0C7
:104AF000282F76EF25F0D890E136E0D7E96E81884F
:104B0000D9D71182120011921200006E0050050DCB
:104B1000F350290FF66EF450F76E100E11B245D017
:104B2000F7220800F550EADF0050050DF350290F79
:104B3000F66EF450F76E100EF722F62A000EF722EA
:104B40000800F550DBDF0050050DF350290FF66E1D
:104B5000F450F76E100EF722020EF626000EF72222
:104B60000800F550CBDF0050050DF350290FF66E0D
:104B7000F450F76E100EF722030EF626000EF72201
:104B80000800F550BBDF0050050DF350290FF66EFD
:104B9000F450F76E100EF722040EF626000EF722E0
:104BA0000800F550ABDF000EA9D7F7220800F5503A
:104BB000FE08A4DF0050050DF350290FF66EF450E7
:104BC000F76E100EF722F62A000EF7220800F550B5
:104BD000FE0894DF0050050DF350290FF66EF450D7
:104BE000F76E100EF722020EF626000EF7220800CE
:104BF000F550FE0883DF0050050DF350290FF66EC7
:104C0000F450F76E100EF722030EF626000EF72270
:104C10000800F550FE0872DF0050050DF350290F13
:104C2000F66EF450F76E100EF722040EF626000E04
:104C3000F7220800F550FE0861DFFE0E5FD7D700AF
:104C4000D96ED7C002F0036AD950520DF3CF00F0ED
:104C5000F4CF01F045EC28F004C0F6FF05C0F7FFE3
:104C60007E0E4CDF520EF36EF46AF350006EF45079
:104C7000016EF306000EF45A01500010D8B411D0A2
:104C8000F750F45C02E1F650F35CD8A004D00001C8
:104C9000D751D8A403D0420E31DFE7D77E0E2EDFE6
:104CA000E4D77E0E2BD7BA000001BE51006EBF5173
:104CB000016EBE07000EBF5B01500010D8B45ED07D
:104CC000BAC0F6FFBBC0F7FF0F0EF76403D00800B1
:104CD000F55005D0F6CFE9FFF7CFEAFFEF50000916
:104CE000D8B422D0BCC0F6FFBDC0F7FF0F0EF764EA
:104CF00003D00800F55005D0F6CFE9FFF7CFEAFF63
:104D0000EF50006EBAC0F6FFBBC0F7FF0F0EF7649E
:104D100003D00800F55005D0F6CFE9FFF7CFEAFF42
:104D2000EF500018D8B424D0BAC0F6FFBBC0F7FFCC
:104D30000F0EF76403D00800F55005D0F6CFE9FF59
:104D4000F7CFEAFFEF50006E016ABCC0F6FFBDC0AE
:104D5000F7FF0F0EF76403D00800F55005D0F6CF2B
:104D6000E9FFF7CFEAFFEF50005E000E015A120094
:104D70000001BA4BBB2BBC4BBD2B96D7006A016A16
:104D80001200CE000001CF51D96E0BD0D906FD0E16
:104D9000E8CF28FA0A0100F000F0282FCBEF26F028
:104DA0000400010ED960F2D7CEC028FA0A0100F043
:104DB00000F0282FD7EF26F01200E16E040ED96E16
:104DC000FA0EE8CF28FA0A0100F000F0282FE4EFED
:104DD00026F00400D92EF4D7E12EF0D71200E16EB0
:104DE000040ED96EFA0EE8CF28FA0A0100F000F09E
:104DF000282FF6EF26F0D92EF5D7E12EF1D71200A5
:104E0000BA00040ED96EFA0EE8CF28FA0A0100F0B3
:104E100000F0282F07EF27F00400D92EF4D7BA0EA0
:104E2000E96E000EEA6EEE06000EED5AEE50ED1041
:104E3000D8B41200E6D7F36E040EE96EFA0EBDDFA9
:104E40000400E92EFBD7F32EF7D71200E96AEA6ACD
:104E50000C6A086A096A0A6A0B6A0450051006108F
:104E6000071006E1046A056A066A076A5AEF28F025
:104E7000C00E0C1606D0D890043605360636073616
:104E80000C2A07AEF8D70C2AD890083609360A360D
:104E90000B360750035C08E10650025C05E1055043
:104EA000015C02E10450005C09E308800450005EEC
:104EB0000550015A0650025A0750035AD89007323B
:104EC0000632053204320C060C503F0BDDE10CBCFF
:104ED000B1EC28F00050046E0150056E0250066ED1
:104EE0000350076E0850006E0950016E0A50026EA2
:104EF0000B50036E0CAE5EEF28F0B1EC28F05EEFC5
:104F000028F00F0E806E816A440E826E3D0E926E06
:104F1000010E936E930E946E010EC26E0E0EC16E54
:104F2000860EC06EC79EC79CC688C696C694C682AB
:104F3000C690C68A0A0EAF6E240EAC6E900EAB6E93
:104F4000F28AD76AD66AD59CD59AD596D584D58269
:104F5000D580F19CF288D08EF28CF28E1200000186
:104F6000F26F0AD0ACA2FED70001F251AD6E120072
:104F70000001F25185EF25F0000E11B0010E026E16
:104F8000036A05D00250EEE0010AF2E0120003507D
:104F9000F9E01200C96EC7A0FED7C9501200E96A35
:104FA000EA6A0050086E0150096E02500A6E035002
:104FB0000B6E026A036A08500402F3CF00F0F4CFCC
:104FC00001F00502F3500126F450022209500402B8
:104FD000F3500126F4500222D8B0032A08500602EA
:104FE000F3500226F450032209500502F350022622
:104FF000F45003220A500402F3500226F450032214
:1050000008500702F350032609500602F350032606
:105010000A500502F35003260B500402F3500326F6
:105020005EEF28F0066A046A056A0250031003E185
:10503000006A016A000C1F0E0612D890062A02367A
:105040000336FCE3033202320250005C0350015885
:1050500004E3016E0250005ED88004360536062E49
:1050600006BAF0D706AE05D0041E042AD8B4050649
:10507000051E0450026E0550036E06AC000C001EA7
:10508000002AD8B40106011E000C066A01AE06D043
:10509000001E004A0106011E068C068E0350800B7E
:1050A000061A03AE13EF28F0021E024A0306031E7F
:1050B00013EF28F0036A026A016A006AE950EA10F5
:1050C00008E003C0EDFF02C0EDFF01C0EDFF00C02E
:1050D000EFFF000CA4000001A4C000F0A5C001F087
:1050E000A5AF1200001E011E002AD8B4012A12002A
:1050F00002500002F3CF04F0F4CF05F00102F350A8
:10510000052603500002F35005261200046E042AFF
:105110000406D8B4000CD8900332023201320032B7
:10512000F7D7046E042A0406D8B4000CD8900036D1
:10513000013602360336F7D7DFC0E1F0E0C0E2F017
:10514000000EE8CFDFF0E8CFE0F0CCEF20F0EECFBC
:1051500000F0EECF01F0EECF02F0EFCF03F0D1EF91
:1051600027F0001E011E021E031E000E002A01224F
:10517000022203221200EECF00F0EECF01F0EECFBC
:1051800002F0EFCF03F028EF27F0EE6AEA50E26278
:0A519000FCD7E950E162F9D71200E4
:020000040030CA
:0C000000FF32F6FEFFF8BBFFFFFFFFFF22
:020000040000FA
:00000001FF
